:100000000C947B000C94A3000C94A3000C943E0D64
:100010000C943E0D0C943E0D0C94A3000C94A30084
:100020000C94A3000C94A3000C94A3000C94130F45
:100030000C94A3000C94A3000C94A3000C94A300B4
:100040000C94F40C0C94A3000C945F0B0C94D40946
:100050000C94A3000C94A3000C94A3000C94A30094
:100060000C94630D0C94A300CD03F403BB030E04A6
:100070002E04620456046204620462049104DD03E7
:10008000130829087A072908CA072908580700070A
:1000900029082908290829082908DA052908B7069E
:1000A0002908440700000000240027002A0000005F
:1000B0000000250028002B000404040404040404A8
:1000C0000202020202020303030303030102040803
:1000D00010204080010204081020010204081020B2
:1000E00000000008000201000003040700000000F7
:1000F00000000000D40F11241FBECFEFD8E0DEBFF8
:10010000CDBF24E0A2E0B2E001C01D92A33FB20740
:10011000E1F712E0A0E0B1E0E2E7FAE202C0059008
:100120000D92A230B107D9F710E0CBE7D0E004C0C0
:100130002197FE010E948D13CA37D107C9F70E948B
:100140005F100C9437150C940000A82FB0E0AB5949
:10015000BB4F9C91292F30E0F901EE0FFF1F2E0FAE
:100160003F1FF901E95CFB4FE081F0E09F01220FA6
:10017000331FE20FF31FEE5EFB4F80818F7B808386
:1001800080916304981306C0992379F0915090935D
:1001900063040BC0882349F0E0916404EF5FE093AF
:1001A0006404F0E0EF5FFD4F90838FEF8C93089530
:1001B0009EEF980F923180F4E82FF0E0DF01A95410
:1001C000BC4F9C91913041F4EE0FFF1FE553FC4F63
:1001D000608371830C941B0C0895CF93863080F557
:1001E000409182025091830221E030E0672B81F43C
:1001F000B90102C0660F771F8A95E2F7CB0180959F
:10020000909584239523909383028093820218C053
:10021000082E02C0220F331F0A94E2F7242B352B3D
:10022000309383022093820290917D04911108C043
:10023000C82F0E94A30CBC018C2FCF910C940E09E7
:10024000CF910895BF92CF92DF92EF92FF920F93DA
:100250001F93CF93DF9300D0CDB7DEB7833008F084
:1002600081C0282F220F220F220F285F253108F08E
:1002700024E1B62EF82EE82EEE0CEE0CEE0C30E05B
:10028000CC24C394E21610F58EEF8E0D8231D8F493
:100290000E2D10E0F801E954FC4F9081923098F453
:1002A000DD24D3948C2D8B2109F4D12C000F111F48
:1002B000913009F043C03C29F801E553FC4F8D2DE6
:1002C00090E091838083CC0CE394DCCFF1100AC0E2
:1002D0003C7FF8948BB1632F609568233B21632B9F
:1002E0006BB92AC081E0F8121AC02B2D2323F89491
:1002F00095B1832F8F7380958923922F9F73892BBC
:1003000085B988B122952695269523703295369524
:100310003695337030958323822B88B90DC03F709A
:10032000F89488B1632F660F660F609568233B21B0
:10033000330F330F632B68B9789414C0DD2009F4B0
:10034000BBCFF801E553FC4F80819181019709F4FF
:10035000B3CF62E08E2D2A8339830E94670C2A81F5
:100360003981AACF0F900F90DF91CF911F910F91FC
:10037000FF90EF90DF90CF90BF9008956F927F92A3
:100380008F929F92AF92BF92CF92DF92EF92FF92A5
:100390000F931F93CF93DF931F92CDB7DEB7982FA4
:1003A0003B01843108F004C1082F10E0F801E95442
:1003B000FC4F8081833009F490C0843009F0F8C08C
:1003C0009250923108F0EDC0F801EB59FB4FE080FC
:1003D000F12C6701CC0CDD1C603282E078070CF058
:1003E00042C077FD05C0653B710524F4DB0104C004
:1003F000A0E001C0A4EBB0E0F601EE0DFF1DE95C4A
:10040000FB4F818128E830E04901881A910887FD77
:100410009394880C991C880C991C092C000CAA0830
:10042000BB08828128E532E0281B310987FD33951E
:10043000220F331F220F331FA901330F660B770BD7
:100440009A01AB01281939094A095B090E94FE1477
:1004500024EB30E040E050E00E94D414820E931E62
:10046000A41EB51E01C04B01F601EE0DFF1DE95C97
:10047000FB4F20812C3008F094C0318188E890E057
:10048000831B910937FD9395880F991F880F991F3A
:100490008816990684F0828148E552E0481B51098C
:1004A00087FD5395440F551F440F551FC401481530
:1004B00059050CF4CA010297880F991F4FB7F89499
:1004C00030E0F901EE0FFF1F2E0F3F1FF901EE5E26
:1004D000FB4F928381834FBF64C0933049F08BEF11
:1004E000890F823028F087EF890F833008F059C0D8
:1004F00061E0892F99830E94670C998161147104CE
:1005000011F460E005C08FEF6816710429F461E012
:10051000892F0E941B0C45C0F801E052FF4FE49167
:10052000E330F9F048F4E130B9F0E230A1F584B5F8
:10053000806284BD68BC35C0E730E9F0E83019F16D
:10054000E43049F580918000806280938000709251
:100550008B0060928A0025C084B5806884BD67BC2A
:1005600020C0809180008068809380007092890014
:100570006092880016C08091B00080688093B000BF
:100580006092B3000EC08091B00080628093B00092
:100590006092B40006C080E8681671040CF0B7CF12
:1005A000B0CF000F111FF801E553FC4F718260823C
:1005B0000F90DF91CF911F910F91FF90EF90DF90FF
:1005C000CF90BF90AF909F908F907F906F90089545
:1005D000DB01909163049C30A8F530916404682F8E
:1005E00070E0332369F0E32FF0E0EF5FFD4F80818F
:1005F000FB01EB59FB4F808331503093640407C0FB
:10060000FB01EB59FB4F90839F5F90936304FB01C9
:10061000EB59FB4F808190E09C01220F331F820F2A
:10062000931F1A161B0634F4141615061CF49A01AF
:10063000AD0104C020E639E040E252E0895C9B4F06
:100640000C94910E4DE251E063E181E70C94250991
:100650008F929F92AF92BF92CF92DF92EF92FF92D2
:100660000F931F93CF93DF931F92CDB7DEB7C82EA2
:10067000D12C960124593C4F4901F901E55BFF4F0C
:1006800090819F3709F44DC1963041F490917C04DC
:10069000992321F06630710509F025C17B01182FDF
:1006A0000EEF080F0231F8F464307105E1F0F60145
:1006B000EB59FB4F80818C30B0F490E0FC01EE0FE1
:1006C000FF1F8E0F9F1FFC01E95CFB4F808190E0B4
:1006D000FC01EE0FFF1F8E0F9F1FFC01EE5EFB4F14
:1006E000808186FD06C192EF910F963068F461E03B
:1006F00070E082E0E816F10411F060E070E0892F0C
:1007000099830E94ED009981023118F5E12FE69559
:10071000E695E695812F8770F0E0E05BFD4FE114F0
:10072000F10421F02BE0E216F10449F421E030E07D
:1007300001C0220F8A95EAF78081282B09C021E0A9
:1007400030E001C0220F8A95EAF7209580812823A6
:1007500020835601AA0CBB1CF501E553FC4F118206
:1007600010823CE0E316F10408F0ACC0F701EC5C49
:10077000FF4F0C948D13963008F0D3C0023120F453
:1007800060E0812F0E94670CF401E55BFF4F8081E0
:100790008F3709F4C6C082E093C0023108F0C1C0AF
:1007A00060E0812F0E94670CF401E55BFF4F8081C0
:1007B0008F3709F4B6C01082B4C0023108F0B1C05E
:1007C00062E0812F0E94670CF401E55BFF4F80819E
:1007D0008F3711F08BE08083F501E553FC4F81E00A
:1007E00090E0918380839DC0023108F09AC0F401AB
:1007F000E55BFF4F8081833021F460E0812F0E9410
:100800001B0C61E0812F0E94670CF401E55BFF4F38
:1008100080818F3709F485C081E052C0133049F0E0
:100820008BEF810F823028F087EF810F833008F043
:1008300078C061E0812F0E94670C61E0812F0E94E7
:10084000670C60E0812F0E941B0CF401E55BFF4FF9
:1008500080818F3709F465C083E032C0023108F02F
:1008600060C0F401E55BFF4F80818F3711F084E0B9
:100870008083F601EB59FB4F80818F3FF1F190E0CF
:10088000FC01EE0FFF1F8E0F9F1FFC01E95CFB4F69
:10089000808190E0FC01EE0FFF1F8E0F9F1FFC0177
:1008A000EE5EFB4F808186FD3CC027C012511230A6
:1008B000C0F5F401E55BFF4F80818F3791F186E051
:1008C00080832FC081E491E00F90DF91CF911F9141
:1008D0000F91FF90EF90DF90CF90BF90AF909F90DF
:1008E0008F900C945E0910927C049FEF909300010E
:1008F000D5CE812F0E94A500F6CE4FEF5FEF6FEFB0
:100900007FEF812F0F90DF91CF911F910F91FF907B
:10091000EF90DF90CF90BF90AF909F908F900C940E
:10092000E8020F90DF91CF911F910F91FF90EF9010
:10093000DF90CF90BF90AF909F908F9008950F93CE
:100940001F93CF93082F10E0F801E05BFD4F9081DB
:10095000C62FC92307581B4F411104C0D8019C91D1
:100960009C1771F1682F80916C0390916D03DC01ED
:10097000ED91FC916F7060690190F081E02D099517
:1009800080916C0390916D03DC01ED91FC916C2FD3
:100990006F770190F081E02D099580916C03909123
:1009A0006D03DC01ED91FC916C2F70E0660F672FF9
:1009B000661F770B0190F081E02D0995F801C08347
:1009C000CF911F910F910895833020F5282F30E0AB
:1009D000F901ED5AFD4F6083672BE1F0F901E05B0F
:1009E000FD4F9081811103C069B16C7F0FC08130D0
:1009F00049F463B136B140E4349F900111246F7320
:100A0000622B04C066B16C7366956695692341E0FC
:100A10000C949F040895CF92DF92EF92FF920F9370
:100A20001F93CF93DF931F92CDB7DEB7082F6B01D3
:100A3000142F6F3F8FEF780709F181E08093AB02AD
:100A40000093CD021092AC021092CE0286E094E0A8
:100A500029830E94E50A2981822F0E947709E0916B
:100A60004E02F0914F02E230F10550F0EE0FFF1F01
:100A7000EE0FFF1F35973197F1F702C0C12CD12C33
:100A80008091AA028111FCCF212F113208F020E2BF
:100A900081E08093AA028093A9029FEF9093A8021D
:100AA0001092A702920F9093A602809385028091E4
:100AB0008502902F990F892B809385028091840263
:100AC000813061F410928402809185028093BB0092
:100AD0008091BC0083FDF8CF85EC01C085EE80934A
:100AE000BC008091AA028130E1F38091A7028217B5
:100AF00010F42091A702A6E8B2E04EE754E0FA0114
:100B00008E2F841B821718F48D918193F9CF109248
:100B10009F0420939E04E12EF12C30E0E216F306B0
:100B20001CF482E591E005C02E153F0524F48FE604
:100B300091E00E945E0900930E02C0920F02C12C48
:100B4000D12CCE14DF0434F490919E0480919F0444
:100B5000981310C062E0610F4EE052E087E70F90FB
:100B6000DF91CF911F910F91FF90EF90DF90CF9089
:100B70000C94250986E094E00E94990AF601E25F50
:100B8000FD4F82838FEFC81AD80ADBCFEF92FF9216
:100B90000F931F93CF93DF9390E0FC01E956F10987
:100BA000E231F10508F055C2EA01162FE05CFF4F73
:100BB0000C948D132981922F987125FF03C08BE827
:100BC00091E05AC0888131E026FB222720F92327B3
:100BD000983069F160F491113CC23093AB0280937C
:100BE000CD021092AC021092CE0202E007C090310A
:100BF00009F43CC0983109F46DC02BC2011778F498
:100C0000FE01E00FF11D8181608120E8829F601963
:100C1000112486E094E00E94E50A0E5FEFCF81E0A8
:100C20000E94770983E191E00197F1F712C24A81AE
:100C30006B81163069F430E8639FB0011124640FB2
:100C4000711D9D814C81E0E89E9F4019112406C0D2
:100C5000F0E86F9F401911246FEF7FEFDF91CF9184
:100C60001F910F91FF90EF900C940B05E091000104
:100C7000E73054F08BEA91E0DF91CF911F910F9113
:100C8000FF90EF900C945E099A814B81663069F475
:100C900030E8439FA0011124490F511D3D819C81E3
:100CA00060E8369F9019112406C0F0E84F9F901914
:100CB00011244FEF5FEFEF5FE093000135E0E302B7
:100CC000F0011124E65AFD4F8083528341839383C0
:100CD0002483BFC120910001121614F08FEF44C08D
:100CE00090E0622F022E000C770B35E0492F50E088
:100CF0006417750774F0349FF001359FF00D1124CF
:100D0000E65AFD4F4081481302C085E026C09F5F30
:100D1000EDCF90E0FACF9830F8F4FA0131968E9F3B
:100D2000D0018F9FB00D1124A65ABD4F3C91849FD6
:100D3000F001859FF00D1124E65AFD4F3083119686
:100D40004D915C9112975283418313963C91139776
:100D5000338314963C9134839F5F492F50E064178E
:100D60007507CCF68FEF820F8093000172C1288146
:100D7000898160E8869FC0011124820F911D009730
:100D800021F090934F0280934E0280917C04811158
:100D900060C1C0E08EEE8C0F823028F466E070E017
:100DA0008C2F0E942803CF5FC431A1F781E080938C
:100DB0007C0410929F0410929E041092AC02109238
:100DC000CE021092AA028093A9021092840261E0DE
:100DD00082E10E941B0C61E083E10E941B0C809168
:100DE000B9008E7F8093B9008091B9008D7F809388
:100DF000B90088E48093B80085E48093BC0029C1E1
:100E0000653008F426C11881F9800A81EB80CC8115
:100E10008EEF810F823108F01CC1E12FF0E0EB5919
:100E2000FB4F20812C30B0F430E0F901EE0FFF1FB2
:100E30002E0F3F1FF901E95CFB4F208130E0F901E3
:100E4000EE0FFF1F2E0F3F1FF901EE5EFB4F80815B
:100E500086FDFBC080E8C89FA00111244E0D511DE6
:100E600090E8099FB00111246F0D711D812F0E9420
:100E7000E80264E070E0812FDF91CF911F910F9124
:100E8000FF90EF900C942803623008F4E2C02881B0
:100E90008981E0E88E9FC0011124820F911D009787
:100EA00011F481E090E09093020180930101D1C0A0
:100EB000623008F4CEC0698170E0123091F08A810E
:100EC000F0E88F9FC0011124682B792B133049F073
:100ED0008B8190E090E4899F902D88271124682BC6
:100EE000792B8881DF91CF911F910F91FF90EF9027
:100EF0000C94BE0180EF0E946A098CE60E946A0988
:100F0000CEEF84EF8C0F863038F482E00E946A09BD
:100F10008AE00E946A0909C0C13039F483E00E9466
:100F20006A0988E00E946A0908C08DEF8C0F823040
:100F3000A8F389EF8C0F833088F3C23130F484E05A
:100F40000E946A098EE00E946A0980EF8C0F82304D
:100F500030F486E00E946A0981E00E946A098FE706
:100F60000E946A09CF5FC23121F1C23150F680E0A0
:100F70000E946A0981E00E946A098BE00E946A0966
:100F800081E00E946A0981E00E946A0981E00E9472
:100F90006A09B7CF662309F45CC0C88180EF0E945C
:100FA0006A098EE60E946A098C2F0E946A09C43180
:100FB00048F087EFDF91CF911F910F91FF90EF9055
:100FC0000C946A09D0E0FE01E954FC4F80810E9434
:100FD0006A09CC0FDD1F8E0105531C4FF80180817B
:100FE0008F770E946A09F801808191819C012078A5
:100FF000232B39F0880F892F881F990B8F770E9438
:101000006A09C553DC4F888199819C012227307C75
:10101000232B79F2990F880B990F982F881F8F77C0
:101020000E946A09C6CF80EF0E946A098AE60E9480
:101030006A09C2EFC63010F48C2F01C08FE70E94FE
:101040006A09CF5FC630B1F7B4CF812F0E94A500E7
:1010500001CFDF91CF911F910F91FF90EF900895F5
:101060000F931F93CF93DF93EC010CE613E0D801AD
:101070008D919C91DC01ED91FC916C2F6F7701902B
:10108000F081E02D0995F80180819181DC01ED91DD
:10109000FC91CC0FCD2FCC1FDD0B6C2F6F77019007
:1010A000F081E02DDF91CF911F910F9109948091F4
:1010B0006C0390916D03DC01ED91FC910190F08146
:1010C000E02D67EF099480916C0390916D03DC0132
:1010D000ED91FC910190F081E02D60EF0994CF93A8
:1010E0000E94630880916C0390916D03DC01ED9187
:1010F000FC910190F081E02D69E7099580916C03E6
:1011000090916D03DC01ED91FC91A0916F03B09182
:1011100070030190F081E02D6C91099580916C0332
:1011200090916D03DC01ED91FC91A0916F03B09162
:1011300070030190F081E02D11966C910995C2E049
:1011400080916E03C81760F4E0916F03F091700313
:10115000EC0FF11D808190E00E943008CF5FF0CF4E
:10116000CF910C945708CF93DF93CCE6D3E08881DE
:101170009981DC01ED91FC910190F081E02D69EF06
:10118000099588819981DC01ED91FC910190F081B4
:10119000E02D62E0099588819981DC01ED91FC9157
:1011A0000190F081E02D65E0DF91CF910994CF921D
:1011B000DF92EF92FF920F931F93CF93DF936C0117
:1011C0007A018B01C0E0D0E0CE15DF0589F0D801AF
:1011D0006D918D01D601ED91FC910190F081E02D92
:1011E000C6010995892B11F47E0102C02196ECCF2E
:1011F000C701DF91CF911F910F91FF90EF90DF908A
:10120000CF9008958FEC92E00E941C0A21E0892B78
:1012100009F420E0822F08950E94C014CF93DF9339
:10122000EB01A0916C03B0916D03ED91FC911197CE
:101230008F70682F606E0190F081E02DCD010995CF
:10124000CE01DF91CF910C943008EF92FF920F9373
:101250001F93CF93DF9300D01F92CDB7DEB7162F29
:101260004A835B8389830E946308A0916C03B091D9
:101270006D03ED91FC9111970190F081E02D898132
:10128000682FCD0109954A81042FE42E5B81F52E4C
:101290008E2D801B811738F4F70181917F0190E03A
:1012A0000E943008F5CF0F900F900F90DF91CF91F3
:1012B0001F910F91FF90EF900C945708FC01019043
:1012C0000020E9F73197BF01681B790BAC0181E77A
:1012D0000C942509A0916C03B0916D03ED91FC91E4
:1012E00011970190F081E02D682FCD010994382FDE
:1012F0002091CE029091CD02213208F049C0809118
:10130000AA028111FCCF42E04093AA023093A902C5
:101310003FEF3093A8021092A7022093A602ADEAF5
:10132000B2E046E852E0FA013E2F341B321718F4BF
:101330003D913193F9CF1092850220918502990F4A
:10134000922B9093850290918402913061F41092D7
:101350008402909185029093BB009091BC0093FD14
:10136000F8CF95EC01C095EE9093BC009091AA0245
:101370009230E1F39091A8029F3F79F08091A8020A
:10138000803241F08091A802803331F084E005C0C2
:1013900081E003C082E001C083E01092AC021092B1
:1013A000CE021092AB0208951F920F920FB60F92C9
:1013B00011242F933F934F935F936F937F938F935A
:1013C0009F93AF93BF93EF93FF938FEC92E00E94B4
:1013D000910BFF91EF91BF91AF919F918F917F9171
:1013E0006F915F914F913F912F910F900FBE0F9092
:1013F0001F901895FC01918D828D981761F0828D58
:10140000DF01A80FB11D5D968C91928D9F5F9F7338
:10141000928F90E008958FEF9FEF0895FC01918DDA
:10142000828D981731F0828DE80FF11D858D90E047
:1014300008958FEF9FEF0895FC01918D228D892FE4
:1014400090E0805C9F4F821B91098F7399270895CC
:1014500080E090E0892B29F00E94020981110C9410
:10146000000008953FB7F8948091EB049091EC044C
:10147000A091ED04B091EE0426B5A89B05C02F3FC6
:1014800019F00196A11DB11D3FBFBA2FA92F982FAA
:101490008827820F911DA11DB11DBC01CD0142E025
:1014A000660F771F881F991F4A95D1F7089585ED1C
:1014B0008093BC008091BC0084FDFCCF1092AA02F6
:1014C00008954091C304262F30E0240F311D2132AE
:1014D0003105DCF42091AA022430C9F4FC0180E03B
:1014E00090E0861758F43091C3042191DC01AF5588
:1014F000BB4FA30FB11D2C930196F3CF8091C30472
:10150000680F6093C30480E0089581E0089582E04D
:1015100008950895E0919F0480919E04E81730F4A7
:10152000F0E0E258FB4F808190E008958FEF9FEF4D
:10153000089590919F0480919E04981750F4E92F8C
:10154000F0E0E258FB4F208130E09F5F90939F04D2
:1015500002C02FEF3FEFC901089580919E0490E0F3
:1015600020919F04821B91090895CF92DF92EF9200
:10157000FF920F931F93CF93DF937C01262F972F1A
:101580008A018091AB02882391F0C62FD72F6E017C
:10159000C40ED51ECC15DD0571F06991D701ED9112
:1015A000FC910190F081E02DC7010995F3CF642FE4
:1015B000822F0E94610AC801DF91CF911F910F9184
:1015C000FF90EF90DF90CF900895CF93DF931F921D
:1015D000CDB7DEB769832091AB022223D1F02091F1
:1015E000CE02203240F021E030E0FC013383228340
:1015F00080E090E015C08091AC02E82FF0E0E35568
:10160000FD4F998190838F5F8093AC028093CE02CF
:1016100005C061E0CE0101960E94610A81E090E080
:101620000F90DF91CF9108950F931F93CF93DF9386
:1016300081E080937D0480917C04882329F01092BE
:101640007C048FEF8093000110925302109250029D
:1016500010927904109254021092510210927A045E
:10166000109255021092520210927B0405E614E08B
:10167000C0E0DFEF82EF8C0F863018F462E070E09C
:1016800006C08EEF8C0F823128F461E070E08C2F61
:101690000E942803F801D1938F01CF5FC43151F725
:1016A00010928302109282021092640410926304DA
:1016B00010927D04DF91CF911F910F9108951F9299
:1016C0000F920FB60F9211242F938F939F93EF9346
:1016D000FF93E091DF02F091E0028081E091E5026A
:1016E000F091E60282FD12C090818091E8028F5F46
:1016F0008F732091E902821751F0E091E802F0E047
:10170000E153FD4F958F8093E80201C08081FF91E6
:10171000EF919F918F912F910F900FBE0F901F907F
:101720001895FC01848DDF01A80FB11DA35ABF4F8E
:101730002C91848D90E001968F739927848FA689D0
:10174000B7892C93A089B1898C9180648C93938DF7
:10175000848D981306C00288F389E02D80818F7DE7
:1017600080830895EF92FF920F931F93CF93DF939F
:10177000EC0181E0888F9B8D8C8D981305C0E889E2
:10178000F989808185FD24C0F62E0B8D10E00F5F56
:101790001F4F0F731127E02E8C8DE8120CC00FB66F
:1017A00007FCFACFE889F989808185FFF5CFCE0162
:1017B0000E94910BF1CF8B8DFE01E80FF11DE35AD2
:1017C000FF4FF0820B8FEA89FB898081806207C01E
:1017D000EE89FF896083E889F9898081806480834C
:1017E00081E090E0DF91CF911F910F91FF90EF90FA
:1017F0000895CF93DF93EC01888D8823C9F0EA899F
:10180000FB89808185FD05C0A889B9898C9186FDF9
:101810000FC00FB607FCF5CF808185FFF2CFA889F6
:10182000B9898C9185FFEDCFCE010E94910BE7CF56
:10183000DF91CF91089590E0FC01E052FF4F349189
:10184000FC01E453FF4F2491FC01E854FF4FE49165
:10185000EE2309F43BC0332339F1333091F038F4EF
:101860003130A9F0323001F584B58F7D12C03730A8
:1018700091F03830A1F03430B9F4809180008F7D40
:1018800003C0809180008F77809380000DC084B565
:101890008F7784BD09C08091B0008F7703C080919D
:1018A000B0008F7D8093B000F0E0EE0FFF1FE25597
:1018B000FF4FA591B4918FB7F894EC91611103C0DB
:1018C00020952E2301C02E2B2C938FBF0895CF93EC
:1018D000DF9390E0FC01E453FF4F2491FC01E854B6
:1018E000FF4F8491882361F190E0880F991FFC01DC
:1018F000EC55FF4FC591D491FC01E255FF4FA591E6
:10190000B491611109C09FB7F89488812095822312
:101910008883EC912E230BC0623061F49FB7F8945A
:101920003881822F809583238883EC912E2B2C93F2
:101930009FBF06C08FB7F894E8812E2B28838FBFF6
:10194000DF91CF9108958E3008F08E5087708064BB
:1019500080937C0080917A00806480937A008091EB
:101960007A0086FDFCCF809178002091790090E08C
:10197000922B08958F929F92AF92BF92CF92DF9257
:10198000EF92FF926B017C010E94320A4B015C01D5
:10199000C114D104E104F104F1F00E94320ADC0127
:1019A000CB0188199909AA09BB09883E9340A10572
:1019B000B10570F321E0C21AD108E108F10888EE00
:1019C000880E83E0981EA11CB11CC114D104E1044F
:1019D000F10419F7DDCFFF90EF90DF90CF90BF902B
:1019E000AF909F908F9008951F920F920FB60F9215
:1019F00011242F933F938F939F93AF93BF93809125
:101A0000560290915702A0915802B091590230911C
:101A1000EA0423E0230F2D3720F40196A11DB11D08
:101A200005C026E8230F0296A11DB11D2093EA04EC
:101A30008093560290935702A0935802B093590294
:101A40008091EB049091EC04A091ED04B091EE0430
:101A50000196A11DB11D8093EB049093EC04A0931B
:101A6000ED04B093EE04BF91AF919F918F913F91A0
:101A70002F910F900FBE0F901F9018951F920F92ED
:101A80000FB60F9211240F900FBE0F901F90189554
:101A9000FC01158216821782DC011896885B9F4F25
:101AA0001D92A817B907E1F71C92DF01A75BBF4F92
:101AB0001D921C92ED56FF4F0190F081E02D309762
:101AC00009F0099408951F920F920FB60F921124F6
:101AD0002F933F934F935F936F937F938F939F9336
:101AE000AF93BF93EF93FF938091B900887F8036C7
:101AF00009F49CC068F5883209F45BC090F4803129
:101B000009F454C038F4882309F4F6C0883009F485
:101B10004DC0F6C0883109F44CC0803209F45DC074
:101B2000EFC0803409F468C048F4803309F455C02C
:101B3000883309F0E5C08093A802D8C0803509F445
:101B40004FC0883509F45DC0883409F0D9C0D6C0CB
:101B5000883909F4C7C0A8F4883709F467C038F495
:101B6000883609F463C0803709F460C0C9C088387A
:101B700009F4B8C0803909F45FC0803809F0C0C0EA
:101B80005BC0803B09F486C038F4803A09F466C033
:101B9000883A09F47FC0B4C0803C09F4A7C0883CEF
:101BA00009F4A4C0883B09F48AC0AAC080918502C8
:101BB00010C09091A7028091A602981770F5E0914D
:101BC000A70281E08E0F8093A702F0E0EA57FD4F55
:101BD00080818093BB0085EC86C08093A8028EC074
:101BE000E091A70281E08E0F8093A7028091BB0055
:101BF000F0E0EA57FD4F80839091A7028091A60202
:101C00006EC0E091A70281E08E0F8093A7028091C1
:101C1000BB00F0E0EA57FD4F80838091A90281115B
:101C20006DC081E08093840284EA61C083E0809388
:101C3000AA021092E704CFCF8091E704803208F027
:101C400051C0E091E70481E08E0F8093E70480911A
:101C5000BB00F0E0E953FB4F8083BDCF85EC809360
:101C6000BC001092AA028091E704803230F4E09127
:101C7000E704F0E0E953FB4F10826091E70470E065
:101C8000E091C504F091C60487EC94E009951092A8
:101C9000E70436C084E08093AA021092C404109234
:101CA000C304E091C104F091C20409958091C3047A
:101CB000811105C081E08093C3041092A104E091DA
:101CC000C40481E08E0F8093C404F0E0EF55FB4F15
:101CD00080818093BB009091C4048091C3049817C5
:101CE00008F479CF85E88093BC000AC085EC809326
:101CF000BC001092AA0204C01092A8020E94570AC7
:101D0000FF91EF91BF91AF919F918F917F916F91D3
:101D10005F914F913F912F910F900FBE0F901F90A9
:101D20001895DF92EF92FF920F931F93CF93DF935B
:101D3000EC01D62E7A01890188818C3008F06AC0C6
:101D400061E08D2D0E94670C8881E82FF0E09F01F3
:101D5000220F331FE20FF31FEE5EFB4F9D2D9F738B
:101D60002081207CD22ED92AD08260E272E0AB01A1
:101D70004E195F0957FF02C04D5F5F4F559547955C
:101D800055954795498340E659E09A01201B310B50
:101D900037FF02C02D5F3F4F359527953595279525
:101DA0002A836CE00E9481139CE0899FB00111247A
:101DB00040E050E09A01260F371FF901EE0FFF1F98
:101DC0002E0F3F1FF901EE5EFB4F908196FD16C06E
:101DD0004F5F5F4F4C30510569F781110FC0109272
:101DE000800082E080938100109285001092840030
:101DF000B19A80916F00826080936F00E881F0E07B
:101E0000CF01880F991FE80FF91FEE5EFB4F80810D
:101E1000806480838881DF91CF911F910F91FF9023
:101E2000EF90DF9008951F920F920FB60F9211243A
:101E30002F933F934F935F936F937F938F939F93D2
:101E4000AF93BF93EF93FF938091A00487FF05C0EA
:101E500010928500109284001BC02091A004022ED5
:101E6000000C330B8091360490E02817390784F476
:101E70008091A004082E000C990BFC01EE0FFF1FAF
:101E80008E0F9F1FFC01EE5EFB4F808186FD15C00B
:101E90008091A0048F5F8093A0042091A004022E63
:101EA000000C330B8091360490E028173907C4F4F6
:101EB0008091A0048C3064F113C08091A004082E9E
:101EC000000C990BFC01EE0FFF1F8E0F9F1FFC01F2
:101ED000EE5EFB4F808160E08F730E941B0CD8CFB9
:101EE0008091840090918500049680349C4918F478
:101EF00080E49CE905C0809184009091850004965F
:101F000090938900809388008FEF8093A0043BC05A
:101F100020918400309185008091A004082E000C4F
:101F2000990BFC01EE0FFF1F8E0F9F1FFC01EE5E51
:101F3000FB4F81819281820F931F90938900809340
:101F400088008091A004082E000C990BFC01EE0F74
:101F5000FF1F8E0F9F1FFC01EE5EFB4F808186FFEF
:101F600012C08091A004082E000C990BFC01EE0F0A
:101F7000FF1F8E0F9F1FFC01EE5EFB4F808161E013
:101F80008F730E941B0CFF91EF91BF91AF919F91B6
:101F90008F917F916F915F914F913F912F910F9012
:101FA0000FBE0F901F901895CF92DF92EF92FF9285
:101FB0001092D2021092D10278EEC72E73E0D72E83
:101FC000E12CF12CC092D302D092D402E092D5023F
:101FD000F092D60281E191E09093D0028093CF02FB
:101FE00085EC90E09093DC028093DB0284EC90E03F
:101FF0009093DE028093DD0280EC90E09093E0020B
:102000008093DF0281EC90E09093E2028093E10202
:1020100082EC90E09093E4028093E30286EC90E0FF
:102020009093E6028093E5021092E8021092E90292
:102030001092EA021092EB0210926E03109270035B
:1020400010926F03109205048CE693E00E94480DF5
:102050001092090410920804C0920A04D0920B0452
:10206000E0920C04F0920D0481E291E09093070459
:102070008093060480913604A7E3B4E09FEF48EB19
:102080005BE08C3078F48C93282F30E0F901EE0F70
:10209000FF1F2E0F3F1FF901EE5EFB4F528341835E
:1020A0008F5F01C09C93139624E0AB35B20749F7CC
:1020B00080933604FF90EF90DF90CF90089578944E
:1020C00084B5826084BD84B5816084BD85B582603D
:1020D00085BD85B5816085BD80916E0081608093EE
:1020E0006E00109281008091810082608093810057
:1020F0008091810081608093810080918000816067
:10210000809380008091B10084608093B1008091C1
:10211000B00081608093B00080917A0084608093E9
:102120007A0080917A00826080937A0080917A00B0
:10213000816080937A0080917A00806880937A0031
:102140001092C10085E180936E0380916F0390919E
:1021500070030E942814C0916E03D0E0CE01019656
:102160000E9493139093700380936F03FC01EC0F14
:10217000FD1F108212E0DC011C9325E011962C93C8
:10218000AE01425051096DEE71E002960E94C514F5
:102190008EEB91E09093F4038093F30382E291E05D
:1021A0009093F6038093F5038DEE90E09093F803FF
:1021B0008093F70384EE94E09093FA038093F903FD
:1021C00088E293E09093FC038093FB0388ED90E01A
:1021D0009093FE038093FD0386EC95E090930404B6
:1021E0008093030484E19BE0909300048093FF03B9
:1021F000E091DF02F091E0021083E091DF02F091C4
:10220000E0021082E091DB02F091DC021082E091AA
:10221000DD02F091DE0280E180831092E702E0911E
:10222000E302F091E40286E08083E091E102F09124
:10223000E202808180618083E091E102F091E2021C
:10224000808188608083E091E102F091E2028081E8
:1022500080688083E091E102F091E20280818F7DCD
:1022600080838FEC92E090936D0380936C03809158
:102270000504811150C061E08DE00E94670C62EDA1
:1022800070E080E090E00E94BA0C61E08DE00E9476
:102290001B0C68E270E080E090E00E94BA0C60E005
:1022A0008DE00E941B0C62ED70E080E090E00E94E7
:1022B000BA0C61E08DE00E941B0C68E270E080E0E7
:1022C00090E00E94BA0C60E08DE00E941B0C6AEF67
:1022D00070E080E090E00E94BA0CC0E062ED70E037
:1022E00080E090E00E94BA0C61E08DE00E941B0C3F
:1022F00068E270E080E090E00E94BA0C60E08DE05F
:102300000E941B0CCF5FC53049F76DE770E080E09D
:1023100090E00E94BA0C0E94B30880916E03811174
:102320000E946F080E94140BBB24B39432E0A32ECA
:1023300015E080915302882349F069B180915002E1
:1023400068236C7F40E080E00E949F0480915402EB
:10235000882379F063B196B1B0E49B9FC00111244A
:102360006F73862B60915102682340E081E00E94E8
:102370009F04809155028823D9F066B16C736695ED
:10238000669580915202682340E082E00E949F049B
:102390000FC080916C0390916D03EC01E881F9818D
:1023A0000680F781E02D09958F3FDFEF9D0771F4DF
:1023B00080916C0390916D03DC01ED91FC910480A0
:1023C000F581E02D0995892B21F71EC1382F209129
:1023D000B403222309F467C0873F09F055C0109267
:1023E000B40380917403813751F0893709F03EC0FE
:1023F00080916E038823E1F20E946F08D9CFE091AB
:102400000104F0910204309799F22091B5033091C4
:10241000B603C901019797FDC90195958795082FC6
:10242000A4E7B3E040E050E030E04E5F5F4F30178C
:1024300070F4BA0164597C4FEB012F812C936885AD
:10244000D0E86D9F201911242D933F5FEECF99277F
:10245000DC01A459BC4F17968C911797882311F073
:1024600018961C9284E793E00995A2CFE0910304AB
:10247000F0910404309709F49BCF6091B50361504B
:1024800045E753E0099594CF2091B5033091B60309
:10249000F901E459FC4F80872F5F3F4F3093B6031B
:1024A0002093B50385CF20917103222309F469C0DD
:1024B00087FD67C09FEF920F90937103E92FF0E0C3
:1024C000E459FC4F8087911173CF80917203882368
:1024D00009F46ECF803D09F445C050F4803901F114
:1024E000803C09F04BC0E091F703F091F8033EC047
:1024F000843F39F1853F51F1803E09F03FC0E091C2
:10250000F303F091F4033097C9F180917403609163
:10251000750370E020E8829F600D711D11242BC0AF
:10252000E091F503F091F603309741F18091740347
:102530006091750370E090E8899F600D711D112412
:102540001AC0E091FB03F091FC0304C0E091FD038D
:10255000F091FE03309791F06091740370E08091E8
:1025600075030BC0E091F903F091FA03309731F055
:102570006091740370E08091730309951092720367
:1025800017CF303F38F4282F207F30E08F708093B2
:10259000730302C09C013327203F310559F17CF4BD
:1025A000203C310511F124F420393105D9F000CF58
:1025B000203D3105D1F0203E3105A1F0F9CE293F73
:1025C0003105F9F034F4C901845F9109029750F0A4
:1025D000EFCE2F3F310509F0EBCE8CE693E00E9461
:1025E000480DE6CEA092710302C0B0927103209311
:1025F0007203DECEB092B4031092B6031092B5030C
:10260000D7CE0E94B308D4CE8FB7F894C0905602AC
:10261000D0905702E0905802F09059028FBFC092BC
:102620005F04D0926004E0926104F09262048091B1
:102630005B0490915C04A0915D04B0915E044091B4
:1026400001015091020160E070E0C81AD90AEA0A5B
:10265000FB0A4C155D056E057F0508F04FC0840F21
:10266000951FA61FB71F80935B0490935C04A093F3
:102670005D04B0935E0487EBE82E83E0F82E02EF52
:102680000630B8F4E7018881823099F480918202A3
:1026900090918302002E02C0959587950A94E2F7E7
:1026A00080FF07C0802F0E94A30CBC01802F0E94D6
:1026B0000E090F5FDFEFED1AFD0A063009F7809172
:1026C000000187FD1BC000E0202F30E08091000159
:1026D000082E000C990B8217930784F0129FF001CB
:1026E000139FF00D1124E65AFD4F61817281248100
:1026F000438180810E940B050F5FE6CF0E94280A6C
:1027000018CE991B79E004C0991F961708F0961B04
:10271000881F7A95C9F780950895EE0FFF1F0590E1
:10272000F491E02D0994CF93DF938230910510F45A
:1027300082E090E0E091F104F091F20420E030E0DA
:10274000C0E0D0E0309711F140815181481759071E
:10275000C0F04817590761F482819381209719F0DE
:102760009B838A832BC09093F2048093F10426C04C
:102770002115310519F04217530718F49A01BE01CB
:10278000DF01EF010280F381E02DDCCF211531055F
:1027900009F1281B390B2430310590F412968D91E4
:1027A0009C9113976115710521F0FB01938382833E
:1027B00004C09093F2048093F104FD01329644C06A
:1027C000FD01E20FF31F81939193225031092D9364
:1027D0003C933AC02091EF043091F004232B41F454
:1027E00020910501309106013093F0042093EF040D
:1027F00020910301309104012115310541F42DB7D9
:102800003EB74091070150910801241B350BE09120
:10281000EF04F091F004E217F307A0F42E1B3F0B36
:102820002817390778F0AC014E5F5F4F2417350742
:1028300048F04E0F5F1F5093F0044093EF048193D4
:10284000919302C0E0E0F0E0CF01DF91CF910895D5
:102850000F931F93CF93DF93009709F48CC0FC0173
:102860003297138212820091F1041091F204011543
:10287000110581F420813181820F931F2091EF0493
:102880003091F0042817390779F5F093F004E093BC
:10289000EF0471C0D80140E050E0AE17BF0750F41C
:1028A00012962D913C911397AD012115310509F137
:1028B000D901F3CF9D01DA013383228360817181D5
:1028C000860F971F8217930769F4EC0128813981DD
:1028D000260F371F2E5F3F4F318320838A819B81D4
:1028E00093838283452B29F4F093F204E093F1045F
:1028F00042C01396FC93EE931297ED0149915991C2
:102900009E01240F351FE217F30771F48081918136
:10291000840F951F029611969C938E9382819381CA
:1029200013969C938E931297E0E0F0E0D8011296F4
:102930008D919C911397009719F0F8018C01F6CFB7
:102940008D919C9198012E5F3F4F820F931F209194
:10295000EF043091F0042817390769F4309729F40F
:102960001092F2041092F10402C0138212821093AA
:10297000F0040093EF04DF91CF911F910F91089520
:1029800081E090E0F8940C943715FB01DC01415094
:10299000504048F001900D920020C9F701C01D92EF
:1029A00041505040E0F70895052E97FB1EF4009427
:1029B0000E94EB1457FD07D00E94061507FC03D0B8
:1029C0004EF40C94EB1450954095309521953F4F63
:1029D0004F4F5F4F089590958095709561957F4F0B
:1029E0008F4F9F4F08950E942815A59F900DB49F6B
:1029F000900DA49F800D911D11240895B7FF0C9494
:102A0000F3140E94F314821B930B0895A1E21A2E73
:102A1000AA1BBB1BFD010DC0AA1FBB1FEE1FFF1F82
:102A2000A217B307E407F50720F0A21BB30BE40BD2
:102A3000F50B661F771F881F991F1A9469F7609519
:102A40007095809590959B01AC01BD01CF010895D3
:102A5000A29FB001B39FC001A39F700D811D1124DF
:102A6000911DB29F700D811D1124911D0895F89440
:022A7000FFCF96
:102A7200FF13000000F304800001000000000000CA
:102A820000B20BD7081C0AFA090E0AF90B00000063
:102A920000E50AB50AAD0A990A8A0A890A4D6178DF
:102AA20020736572766F7320617474616368656404
:102AB20000556E6B6E6F776E2070696E206D6F645D
:102AC20065004932433A20546F6F206D616E792060
:102AD200627974657320726563656976656400491D
:102AE20032433A20546F6F206665772062797465AD
:102AF200732072656365697665640031302D6269A1
:102B0200742061646472657373696E67206E6F749A
:102B120020737570706F7274656400746F6F206DCE
:102B2200616E792071756572696573002F557365E1
:102B320072732F6E6F6F706B61742F446F63756D5C
:102B4200656E74732F41726475696E6F2F53746171
:102B52006E646172644669726D6174612F5374614F
:102B62006E646172644669726D6174612E696E6F22
:022B7200000061
:00000001FF
